:0300000002082EC5
:0C082E00787FE4F6D8FD7581570208754C
:0F0AA9008F907F017E00120AB8D2A67F017E00D7
:100AB800EF1FAC0670011E4C600D0000007D0B7C22
:070AC800BEDCFEDDFC80E94D
:010ACF002204
:08000300C2A7120AA9C2A6223D
:080BA000D2A7120AA9C2A62285
:020A80008F08DD
:100A8200E4F509ED7006E50824808004E50824C039
:100A9200FF12000312077EFF600C120BA0740129E3
:060AA200F9E43AFA80EECF
:010AA800222B
:100A54007F38120003120AB47F0C120003120AB486
:100A64007F06120003120AB47F01120003120AB4B3
:0C0A74007F801200037F017E00020AB8A0
:100B5300AE0753060F530501ED7003EE8003EE2439
:080B6300404480FF1200032250
:080BA800120B53AF03020BA076
:100A21005825644825644425645A0D0A00205765F9
:100A31006C636F6D6520746F207573650054656D0F
:100A4100703A0048756D693A0041004C3A00483AE5
:030A5100004D0055
:1009290001560001243C012350015105C10A102937
:1009390000000000000000000000000000000000AE
:10094900015500015446022703E8C10DC1090153AD
:1009590000C10C023E0000012200015200C10B013E
:060969005700022500000A
:1008BA00750B00750C00750D54750E027B007A00DD
:1008CA007955120558EF7056E55475F00A842430AC
:1008DA00F540E55475F00A84E5F02430F541754297
:1008EA0025E55575F00A842430F54BE55575F00A6F
:1008FA0084E5F02430F54C754DDF754E43750BFFDA
:10090A00750C0A750D2185550E85540F7B007A00EA
:0F091A0079291200827B007A007929120B1B22A7
:100B6B00D3EF9400EE64809480400B7D6EDDFEEF3E
:060B7B001F70ED1E80EA70
:010B81002251
:10067400E5B054F8FF64F87003020758E5226003FC
:1006840002075B752201EF2488700302074F24C020
:10069400607324E0602924F0600D24F860030207ED
:1006A4005BB20DC2098014300D0302075B0556D3FB
:1006B400E55664809483500302075BE4F5562230C8
:1006C4000D0302075BE556B4010E0524D3E524644B
:1006D4008094DC4003E4F524E556B4020E0523D3EC
:1006E400E523648094DC4003E4F523E55664037059
:1006F40066C3E5289406E5279427505B746425288F
:10070400F528E48041200D4FE556B4010E1524C3AD
:10071400E52464809480500375245CE556B4020E8D
:100724001523C3E52364809480500375235CE55648
:10073400B40324D3E5289464E52794004019749CF9
:100744002528F52874FF3527F52722300D09A20A3C
:07075400B3920A22E4F52232
:01075B00227B
:10000E005389F0438901E4F58A758C70C28DD28CC8
:05001E00D2A9D2AF22BF
:03000B00020AF7EF
:100AF700C0E0C0D075D000C007758A00758C70053E
:100B070052120674300A04C2A38002D2A3D007D0BF
:040B1700D0D0E03228
:100B380053877F75985053890F438920758BFD75AE
:0B0B48008DFDC2ABD28ED2AFD2AC222A
:1009AF008B0B8A0C890DAE02AF01EF4E602AC2ACE1
:1009BF00EDD394004020AF051DEF601AAB0B050D72
:1009CF00E50DAA0C7002050C14F912077EF599308B
:0909DF0099FDC29980E0D2AC221E
:100B1B008B088A09890AAE02AF01EF4E600E120BE9
:0D0B2B0082AD07AB08AA09A90A1209AF2282
:030023000209E8E7
:1009E800C0E0C0D0309829859957E55724DC6010BD
:1009F80024FE601024FC601324EA7014C20D8010D9
:100A0800D20D800C300D09D20A8005300D02C20AC1
:090A1800C298C299D0D0D0E0329E
:1003820012000E120A547BFF7A0A792EE4FDFF1244
:100392000A807FE87E03120B6B7F011200037F64E9
:1003A2007E00120B6B1208BA7F327E00120B6BD2E8
:1003B200A4120B380552E552D3941440F7E4F552D7
:1003C2001208BA300D030204F820090ED2097F0187
:1003D2001200037F0A7E00120AB8E5566003020487
:1003E200827BFF7A0A793EFDFF120A807B007A0047
:1003F200794BE4FD7F05120A807BFF7A0A79447DFE
:1004020001E4FF120A807B007A0079407D017F05BA
:10041200120A807BFF7A0A794A7D017F0F120A80D5
:10042200AF24EF3395E0FEAD547C00C3ED9FEE6444
:1004320080F87480985007D20AC2A30204F8D3ED60
:100442009FEE6480F8EC648098401BAF23EF3395F5
:10045200E0FEC3ED9FEE6480F8EC6480985007D212
:100462000AD2A30204F8AF23EF3395E0FED3ED9F47
:10047200EE6480F8EC648098407CC20AD2A3807655
:10048200E52475F00A12075C2430F546E52475F080
:100492000A12075CAFF0EF2430F54775482575491D
:1004A20020E52375F00A12075C2430F539E523753F
:1004B200F00A12075CAFF0EF2430F53A753B257570
:1004C2003C207BFF7A0A794CE4FD7F09120A807B8B
:1004D200007A007946E4FD7F0B120A807BFF7A0ADC
:1004E200794F7D017F09120A807B007A0079397D7C
:1004F200017F0B120A80200D030203B620090ED2DF
:10050200097F011200037F0A7E00120AB8E55660D5
:10051200030203B67BFF7A0A793EFDFF120A807B53
:10052200007A00794BE4FD7F05120A807BFF7A0A8C
:1005320079447D01E4FF120A807B007A0079407DD4
:10054200017F05120A807BFF7A0A79527D017F0FB3
:06055200120A800203B64C
:040BB6007F0CDFFED3
:010BBA002218
:080B97007F247ED9DEFEDFFCA5
:010B9F002233
:050BB000007F14DFFED0
:010BB500221D
:10097000E4FEFCE4FD20A00B000DEDD394FA40F55D
:100980007F6422E4FD120BB630A009EE25E0FE43A1
:1009900006018006EE25E0FE800E30A00B000DED76
:0E09A000D394FA40F57F64220CBC08C7AF0662
:0109AE002226
:060558008B088A09890AE4
:10055E00E4FDF50FF9F510FBFC00C2A000120B979D
:10056E00D2A000120BB60030A00302066E20A00B24
:10057E00000DEDD394FA40F57FFF22E4FD120BB08F
:10058E0020A0FD000DEDD394FA40037FFF22C2AFF1
:10059E001209708F0F120970A9071209708F1012AD
:1005AE000970AB07120970AC07D2AFAF01E50F2F80
:1005BE00FFE433FEE5107583002FFFE5833EFEADAD
:1005CE0003ED7A002FFFEA3EFEAD04ED6F7001EEF3
:1005DE00600FE50F6464700302066BE510646460DF
:1005EE007CE50E64017050E51075F00A842430AB82
:1005FE0008AA09A90A120797E51075F00A84E5F012
:10060E002430AB08AA09A90A9000011207A9E50F28
:10061E0075F00A842430AB0BAA0CA90D120797E5CE
:10062E000F75F00A84E5F02430AB0BAA0CA90D90DF
:10063E0000011207A9802CE510D394325025E50F46
:10064E00C3945F501EAB08AA09A90AE510120797BA
:10065E00AB0BAA0CA90DE50F12079780067FFF22A0
:05066E007FFF227F0068
:010673002264
:10083A00020382E493A3F8E493A34003F68001F24F
:10084A0008DFF48029E493A3F85407240CC8C333BF
:10085A00C4540F4420C8834004F456800146F6DF8E
:10086A00E4800B0102040810204080900929E47EEC
:10087A00019360BCA3FF543F30E509541FFEE49383
:10088A00A360010ECF54C025E060A840B8E493A34A
:10089A00FAE493A3F8E493A3C8C582C8CAC583CA75
:1008AA00F0A3C8C582C8CAC583CADFE9DEE780BE2D
:01096F000087
:10075C00C2D530F707B2D563F0FF05F030E70CB225
:10076C00D5F4048463F0FF05F080018430D502F4E5
:02077C00042255
:10077E00BB010689828A83E0225002E722BBFE0279
:09078E00E32289828A83E49322AC
:10079700BB010689828A83F0225002F722BBFE0141
:0207A700F3223B
:1007A900F8BB010DE58229F582E5833AF583E8F086
:1007B900225006E92582C8F622BBFE05E92582C832
:0207C900F2221A
:10002600E517240BF8E60517227808300702780B47
:10003600E475F0011207F802077E2000EB7F2ED24E
:10004600008018EF540F2490D43440D4FF30040BB2
:10005600EF24BFB41A0050032461FFE518600215AF
:1000660018051BE51B7002051A30070D7808E475A4
:10007600F0011207F8EF020797020AD07403D207BD
:100086008003E4C207F5178B088A09890AE4F51884
:10009600F51AF51BE51860077F2012006180F575DB
:1000A60019FFC201C200C202C203C205C206C208CB
:1000B60012002FFF700D3007057F00120072AF1B74
:1000C600AE1A22B4255FC2D5C20412002FFF24D077
:1000D600B40A00501A75F00A781830D50508B6FF2C
:1000E6000106C6A426F620D5047002D20380D924C0
:1000F600CFB41A00EF5004C2E5D204020272D20154
:1001060080C6D20080C0D20280BCD2D580BAD205C9
:1001160080B47F201200612002077401B5180040E8
:10012600F1120026FF12006102009AD208D2068060
:1001360095120026FB120026FA120026F94A4B7089
:100146000679437A037BFF20022EE518602A7E009B
:100156008E827583001207CB60060EEE651970F06D
:10016600C2D5EBC0E0EAC0E0E9C0E0EE1202B9D0C9
:10017600E0F9D0E0FAD0E0FB12077EFF60AAEBC000
:10018600E0EAC0E0E9C0E0120061D0E02401F9D065
:10019600E03400FAD0E0FBE5190460DCD519D9801B
:1001A600877BFF7A0279B5D202809C79108002792A
:1001B60008C206C2088008D2D5790A8004790AC224
:1001C600D5E519047002F519E4FAFDFEFF120026C2
:1001D600FC7B08200113120026FD7B1030000A125A
:1001E6000026FE120026FF7B20EC3382D592D550E6
:1001F60013C3E43000069FFFE49EFEE42001039D46
:10020600FDE49CFCE4CBF8C201EC700CCFCECDCC67
:10021600E824F8F870F38017C3EF33FFEE33FEEDF2
:1002260033FDEC33FCEB33FB994002FB0FD8E9EBD3
:10023600300105F8D0E0C448B201C0E00AEC4D4EEA
:100246004F78207B0070C2EAB5190040BCC0E012AE
:1002560002BBD0F0D0E0200104C4C0E0C4B201C0AB
:10026600F012004AD0F0D5F0EB02009A120808010D
:10027600375301B15801084C01044201B54F01BD85
:0F0286004401BD49011D4301C35501A74601A70E
:100295004501A747036350010C2D01102E01332B97
:1002A500011423013120034C2A00CC480000012B06
:1002B5003F3F3F00790AA2D5200314300509B91044
:1002C500020404B9080104A2D52006025001042045
:1002D50002689202B518005034C0E07F203003193F
:1002E5007F30A20272067205500F120312C202C2BB
:1002F50006C205C2087F30800F300503E9C0E01251
:100305000061300503D0E0F9D0E0B518CC30051711
:100315007F30B9100C1200617F583004077F788058
:1003250003B908031200613002057F2D0200617FC9
:10033500202008F87F2B2006F322920280CF286E1A
:10034500756C6C2900D2011200263001F8C20178C3
:100355001830D50108F60200CC2D5043495812003B
:10036500262403B405004001E490035E9312005275
:0D037500743A120052D2037518040201B14F
:100B8200E4FFFE12077E600C0FEF70010E09E970A0
:050B9200F20A80EF22D1
:1007CB00BB010CE58229F582E5833AF583E02250E3
:1007DB0006E92582F8E622BBFE06E92582F8E2222D
:0D07EB00E58229F582E5833AF583E4932247
:1007F800FAE6FB0808E6F925F0F618E6CA3AF62202
:10080800D083D082F8E4937012740193700DA3A37F
:1008180093F8740193F5828883E473740293686093
:06082800EFA3A3A380DF93
:100AD000EFB40A07740D120ADB740A309811A89952
:100AE000B8130CC2983098FDA899C298B811F63086
:070AF00099FDC299F599225E
:00000001FF
